:020000040000FA
:02000000040AF0
:080008009F0C0200080C060029
:10001000130A4B0C2800F90C29000000E9020D0A14
:10002000E8020B0A0008000C26006606330A260CBC
:10003000260009090909090909090909090909091C
:100040006606330A0909090909090909090909099B
:1000500009096606330A240C26000909220C260029
:10006000090966072B0A210C26000909200C260025
:100070000909010C26000909000C26000909010CD8
:1000800026000909000C260009096607170A110C49
:10009000260009090909010C2600090909090909AD
:1000A0000909090909096607170A09090909090956
:1000B000090909090909090909096607170A090946
:1000C0000909090909090909090909090909660745
:1000D000170A090909090909090909090909090981
:1000E00009096607170A0909090909090909090916
:1000F0000909090909096607170A09090909090906
:10010000090909090909090909096607170A100CEB
:10011000260009090909090909090909090909093B
:1001200009096607170A000C2600090909090909C7
:10013000090909090909090909096607170A870A46
:021FFE00EA0FE8
:00000001FF
